:020000040000fa
:08000000407f04000100000034
:020000040000fa
:1002000000000000000000000000000000000000ee
:1002100000000000000000000000000000000000de
:1002200000000000000000000000000000000000ce
:1002300000000000000000000000000000000000be
:020000040002f8
:10fe8000af88200080792200000188000000000077
:10fe900000002800601088000040200070108800da
:10fea000a0002000a010880000002800b0108800ea
:10feb00000402000c0108800a0002000f010880042
:10fec00081052000d1108800048020003300070045
:10fed000114cb10040003a0012c7b30082108800f4
:10fee000b2c4b300821088008006eb0004802000ba
:10fef000e1032000d1108800460020002700070001
:10ff0000d11088000603e900fcff3a000c40800095
:10ff10001340800093018800160620001f00070090
:10ff2000d11088000603e900fcff3a000d00e00054
:10ff300003003200e2c4b30082108800eaff3700f9
:10ff4000000ebb00100424000060fe000a00070041
:10ff5000448020001f00080003000000345ebb0046
:10ff60003456bb0034cebb000c86e80010002400e1
:10ff700001000700daff3700003b88005005200031
:10ff8000303b8800a00a2000303b880061e7a800d1
:10ff9000000000000000000000000600aa0220008f
:10ffa0000b0020000e02ae0004003700911080000c
:10ffb000015a78008dc64000000006000060fe0077
:10ffc0008b05e900f7ff3a000a05e900f4ff3a0063
:10ffd000e1022000d11088000c22ef00a4ff3700be
:0cffe0004d650000736100006a21000004
:020000040000fa
:10000800fe7f0100fe7f0100fe7f0100fe7f0100f0
:10001800fe7f0100fe7f0100fe7f0100fe7f0100e0
:10002800fe7f0100fe7f0100fe7f0100fe7f0100d0
:10003800fe7f0100fe7f0100fe7f0100fe7f0100c0
:10004800fe7f0100fe7f0100fe7f0100fe7f0100b0
:10005800fe7f0100fe7f0100fe7f0100fe7f0100a0
:10006800fe7f0100fe7f0100fe7f0100fe7f010090
:10007800fe7f0100fe7f0100fe7f0100fe7f010080
:10008800fe7f0100fe7f0100fe7f0100fe7f010070
:10009800fe7f0100fe7f0100fe7f0100fe7f010060
:1000a800fe7f0100fe7f0100fe7f0100fe7f010050
:1000b800fe7f0100fe7f0100fe7f0100fe7f010040
:1000c800fe7f0100fe7f0100fe7f0100fe7f010030
:1000d800fe7f0100fe7f0100fe7f0100fe7f010020
:1000e800fe7f0100fe7f0100fe7f0100fe7f010010
:0800f800fe7f0100fe7f010004
:020000040000fa
:10010800fe7f0100fe7f0100fe7f0100fe7f0100ef
:10011800fe7f0100fe7f0100fe7f0100fe7f0100df
:10012800fe7f0100fe7f0100fe7f0100fe7f0100cf
:10013800fe7f0100fe7f0100fe7f0100fe7f0100bf
:10014800fe7f0100fe7f0100fe7f0100fe7f0100af
:10015800fe7f0100fe7f0100fe7f0100fe7f01009f
:10016800fe7f0100fe7f0100fe7f0100fe7f01008f
:10017800fe7f0100fe7f0100fe7f0100fe7f01007f
:10018800fe7f0100fe7f0100fe7f0100fe7f01006f
:10019800fe7f0100fe7f0100fe7f0100fe7f01005f
:1001a800fe7f0100fe7f0100fe7f0100fe7f01004f
:1001b800fe7f0100fe7f0100fe7f0100fe7f01003f
:1001c800fe7f0100fe7f0100fe7f0100fe7f01002f
:1001d800fe7f0100fe7f0100fe7f0100fe7f01001f
:1001e800fe7f0100fe7f0100fe7f0100fe7f01000f
:0801f800fe7f0100fe7f010003
:020000040000fa
:020000040002f8
:10ffec00000800008a000000000000000000000073
:020000040000fa
:020000040002f8
:04fffc000000fe0003
:00000001FF
